:020000040000FA
:060000000219FD02031CC1
:03000B0002008D63
:03001300020535AE
:03001B0002009050
:03002B000202D1FD
:03005B0002054457
:030073000203097C
:100080000406080C10182030406080A0C0054032E3
:10009000C2AFC2A853E6EFC28E856B8BC0D0D2D35D
:1000A000C0E0C0F0C2CAA8CCA9CDD2CAD2AF758A6E
:1000B00000C3E8956CF8E9956DF9C3E913F9E81305
:1000C000F8E5666007C3E913F9E813F8E97025E875
:1000D000956E4020956E501CE582B410177C007B15
:1000E000007A007908900000A86AE5667004C3E809
:1000F00013F801FD900000D2A8D2AA61E7E0FDC389
:100100009CC39840EF98EB33FB0582E0FCC39DC392
:100110009840E198EB33FB0582E0FDC39CC3984017
:10012000D398EB33FB0582E0FCC39DC39840C59890
:10013000EB33FB0582E0FDC39CC39840B798EB33DB
:10014000FB0582E0FCC39DC39840A998EB33FB05F7
:1001500082E0FDC39CC398409B98EB33FB0582E093
:10016000FCC39DC398408D98EB33FB0582217890AA
:100170000000D2A8D2AA61E7E0FDC39CC39840EF7B
:1001800098EA33FA0582E0FCC39DC39840E198EAFF
:1001900033FA0582E0FDC39CC39840D398EA33FA52
:1001A0000582E0FCC39DC39840C598EA33FA0582F6
:1001B000E0FDC39CC39840B798EA33FA0582E0FC9F
:1001C000C39DC39840A998EA33FA0582E0FDC39C19
:1001D000C398409B98EA33FA0582E0FCC39DC3981C
:1001E000408D98EA33FA0582EBC46B6A54F0F9EA61
:1001F000C454F0C3996009900000D2A8D2AA61E764
:10020000EBF4C454F0F9EAF4C4540F49FAEBF4C423
:10021000540FFBC3EAF99460FAEB9400FB5020C33F
:10022000E97B007A0079006016C3135006F9C39584
:1002300052600AE9F5527553007900800205533087
:100240003A27C3EA94D0F8EB9407F9400BE8FAE9AF
:10025000FB203509D235415D303502C235203902E7
:10026000B235C3EA33FAEB33FBEB2B3B3BF9C3EB81
:1002700013FBEA13FAEA29FAEB3400FB30E3047AC1
:10028000FF7BFFE5255403601B202A18E55D33F949
:10029000EB7007C3E99A4002E9FAE53CC4332AFA55
:1002A000EB3400FBC3EA33C4540FF8EB33C454F00F
:1002B00048F87005EA60027801900000D2A8D2AA3E
:1002C000E5226002152281D4900000D2A8D2AA6152
:1002D000E7C0D0C0E0C2CF0541E5666009E56560D2
:1002E000057565006104756501E52360021523C38A
:1002F000E55460057555006104E5552401F5555038
:10030000037555FFD0E0D0D032C2AF53E67F75926F
:10031000FA7593FFC22053917FD2AF32C0E0E58AD5
:10032000303408856B8BF0A3D0E032D0E0C2AF53FD
:10033000E6EFC0D0C0E0C0F0D2D3D2AF5388EFA870
:100340008AA98CAA40308D010A758A00758C0075C7
:100350004000438810E566700AC3E833F8E933F9D2
:10036000EA33FA30331FE8C4540FFAE9C454F04AB0
:10037000FAC3132AFAC3E833F8E933F9E82AFAE9A9
:100380003406FB61D830320FC3E833E933FAE82A88
:10039000FAE93400FB61D8303115E875F056A4AAAB
:1003A000F0E975F056A42AFAC5F03400FB61D8C311
:1003B000EA13FAE913F9E813F8E875F056A4AAF07D
:1003C000E975F056A42AFAC5F03400C313FBEA130A
:1003D000FAC3EB13FBEA13FAC3EB94125009C3EA16
:1003E0009434EB940750160522E52270021522C3BF
:1003F000E52294325002A128755400A12BE5226019
:100400000215223036067C007D088117AC31AD32F2
:10041000303A04AC33AD34C3EA9CFAEB9DFB92084E
:10042000AE60AF61303A425007203509D235813590
:10043000303502C235303504AE62AF63203902B2C6
:1004400035C3EA33FAEB33FBA208500AEAF424017D
:10045000FAEBF43400FBC3EA9450FAEB9400FB503F
:100460001478007A007B008175A208500878007A21
:10047000007B0081D4E5255403601B202A18E55D2C
:1004800033F9EB7007C3E99A4002E9FAE53CC4335B
:100490002AFAEB3400FBEA8EF0A4F9AAF0EB8EF016
:1004A000A42AFAC5F03400FBC3EB13FDEA13F8C32A
:1004B000ED13FDE813F80FEF146004C3E833F8C33D
:1004C000E933EA33FAEB33FBDFEDEB30E30678FF99
:1004D0007AFF7B078854D230E86003755500C3E586
:1004E0005BFC955C4002AC5CC3EC95545008EC7529
:1004F000F008A4FAABF0EAF4F8EBF45407F9C3E817
:10050000948CFAE99400FB50047A007B00885689A9
:10051000578A588B5975230AD0F0D0E0D0D053F7C2
:10052000DF43F74043E6103275230AD0F0D0E0D025
:10053000D043E61032C2AAD28EC2CA85CC6C85CD19
:100540006DD2CA32C2AFC0D0C0E0D2D3A8F9E55A4A
:1005500030E20AE5FA20E23520E132A165E5FA3021
:10056000E22B20E128C3E55713F8E55613F5FB8885
:10057000FCC3E55913F8E55813F5E988EA85575A9D
:1005800053F7BFD2A8303402D2AA53E6EF53F7DFB5
:10059000D0E0D0D0D2AF32790180147903801079C5
:1005A0000A800C791E80087964800479C8800078FC
:1005B00017E4D5E0FDD8FAD9F62278FF202828796B
:1005C000A1E76023E548601F74FF8548F084853FFC
:1005D000F030290375F005A4F8C5F0600278FFC378
:1005E000E8955D5002A85D885C22C3E54794A0E5CC
:1005F000489400E55C500314A1FB046002F55C2202
:1006000075E89022055EC3E55E9408405330EDF432
:10061000A8BDA9BE755E00E9FA79A0E76041EA705D
:1006200006E55F6018800CC3E8955F600EE55F50DB
:1006300005600A1480070460FA8002E55FF55FC375
:100640009569401B755BC0C394044013755B80C300
:100650009404400B755B40C394044003755B002217
:10066000E55B2410500274FFF55B22743279A68793
:10067000F0A4C5F0A2F733F55D227547007548F088
:1006800022C2AFC2CAA8CCA9CDAA4130CF010AD29A
:10069000CAD2AFC3EA13FAE913F9E813F8AB42ACD4
:1006A0004388428943C3E89BF8E99C20280A547F89
:1006B000F9302C02E19FC1F8AD448A44F9EA9D5417
:1006C0007FFA600678FF79FFC1DDAE45AF468B4506
:1006D0008C46A842A943C3E89EF8E99FF9C3E548C0
:1006E00013FBE54713FAE82AF547E93BF5485006BE
:1006F0007547FF7548FFE145AA47AB48AC47AD4891
:100700007E047F02C3EB9404400D1E1FC3EB9408CC
:1007100040052029021E1FC3ED13FDEC13FCDEF77C
:10072000C3EA9CFAEB9DFBEF6009C3E913F9E813F8
:10073000F8DFF7EA28FAEB39FB8A478B4850067B4B
:10074000FF8B478B48C3EB94025002D22C30280415
:100750007F03E1707892E6FFC3E53D948240110F7C
:10076000C3E53D94A040010FC3EF940640027F050E
:100770007E02E548C4540FF9E548C454F0F8E54753
:10078000C4540F28F8C3E89EFAE99400FB4009C35B
:10079000EA9401EB940050047A01E4FB0207EBAA0F
:1007A00047AB48EBC4FEEAC4540F4EFCC3EA9CFAC4
:1007B000EB9400FBC3E813C313F8EA28FAEB340008
:1007C000FB8A478B48C3EB94024002C22C7802EBB1
:1007D000C4FE7B00EAC4540F4EFAC3EA98FA4005FF
:1007E000C3940150027A017892E6FF302002E1EBD7
:1007F000854E92854F93D22043E680C3E49AF8E475
:100800009BF9C3E833F8E933F9302C03020880E898
:10081000FAE9FBD3E913FDE813FC884E894FC3EFD7
:1008200094036038EF20E00CE82CF8E93DF9ECFA8D
:10083000EDFB8013E828F8E939F9C3E82401F8E969
:100840003400F97AFF7BFFC3EF9403400F8A508B8B
:1008500051884A894B8C4C8D4D0208B5885089517E
:100860008A4A8B4B8C4C8D4D3028127550F0755147
:10087000FF754CF0754DFF754EF0754FFF0208B5D2
:10088000E8FAD3E813FC884EC3EF94036021EF200D
:10089000E007E82CF8ECFA01A0E8282401F87AFF38
:1008A000C3EF940340098A50884A8C4C0208B588EB
:1008B000508A4A8C4C30200201B5753A02D220434E
:1008C000E680E5255403602DA847A948C3E913F93C
:1008D000E813F8302804E92440F9C2AF53E67F75E5
:1008E0009100C3E498F594E499F595759104D220AC
:1008F00043E680D2AF22D221754900752000302B0B
:10090000037520402114D221754900752040302BF9
:100910000375200078017901202C20E5255403601F
:1009200002C2217914E548C313700104F8C394147A
:1009300040027814302804781B791BC3E833F8C3CD
:10094000E933F9202010E549600C302803D53A043A
:10095000D22221C811BD0549E59BF45440B52002BF
:1009600021B230280908C3E8994001182143202109
:100970000A08C3E899400221142143C22153E67FAB
:10098000759100302C117594007595F0759104D215
:100990002043E680020914E5487EFFC3334009C3C3
:1009A000334005C3334001FEC3E49E759400F595C2
:1009B000218CC3E539940150022114302102211405
:1009C000D80221C62143C222C2AF53E67F759100EF
:1009D000855094855195759104854A92854B93D2A3
:1009E0002043E680D2AFE5255403600720290205A5
:1009F00039801030220D202B0A2021071581158106
:100A00000213CF2278003021027801E53D75F0070E
:100A1000A4F9E5F028F5F0E9A2F013A2F113A2F28F
:100A200013F53DC394785003753D78C3E53D953E7D
:100A30004009C290C292C29475D53F302002413B1A
:100A4000854C92854D93D22043E68022203810C2F7
:100A5000AFD293C29175D50FD2AF759F03611CC2FF
:100A6000AFD293C29575D53CD2AF759F03611C2060
:100A70003810C2AFC29475D533C291D2AF759F13EF
:100A8000611CC2AFC29075D533C295D2AF759F239A
:100A9000611C203810C2AFD291C29575D533D2AF48
:100AA000759F238077C2AFD295C29175D533D2AFEF
:100AB000759F138067203810C2AFC29275D53CC2B3
:100AC00095D2AF759F038054C2AFC29275D50FC245
:100AD00091D2AF759F038044203810C2AFD295C227
:100AE0009375D53CD2AF759F138031C2AFD291C2FE
:100AF0009375D50FD2AF759F238021203810C2AFD8
:100B0000C29075D50FC293D2AF759F23800EC2AF2E
:100B1000C29475D53CC293D2AF759F13227A147BD1
:100B20007880127A107B8C800C7A0D7BB480067AE8
:100B30000B7BC88000E564D5E001227902E4D29302
:100B4000D5E0FDD292D5E0FDC292D5E0FDC293D5AD
:100B5000E0FDE920E002D29030E002D294E564D5D5
:100B6000E0FDE920E002C29030E002C2947496D524
:100B7000E0FDD9C9EAF8D5E0FDD8FBDBB8D2932275
:100B8000C290C292C294D291D293D29575D53F228F
:100B9000788076FF0876FF0876FF0876FF0876FFF4
:100BA0000876FF0876090876FF087601788C7601CA
:100BB0000876FF0876FF0876FF0876FF0876FF08BC
:100BC00076030876FF0876FF0876FF087625087614
:100BD000D00876280876500876040876FF08760252
:100BE0000876FF08767A0876FF0876070876010807
:100BF00076FF0876FF08760008760022FA75F00C7A
:100C0000A4ABF0EAC333F8740133F9E8C333F8E96D
:100C100033F9E8C32BF8E93400F9E8C333F8E933D2
:100C2000F9227888E6C39403D23A5002C23AC23815
:100C3000E630E102D238A23892397886E614900084
:100C4000809378A6F67886E6F53FC3940250037544
:100C50003F02789CE6753EFFB40203753EA0B403E4
:100C600003753E8278A0E6F8600674282409D8FC53
:100C7000F5697896E671FC88318932789EE671FCD8
:100C8000883389347897E671FC88358936718022FB
:100C90003036117A007B007CFF7D007E0091F68B60
:100CA000618A6022303A227896E6FA7B00789EE6E6
:100CB000FC7D00C3EA33FAEB33FBC3EC33FCED33CA
:100CC000FD7E0A91F68B638A627896303A02789EAE
:100CD000E6FA7B007897E6FC7D007E00303A10C390
:100CE000EA33FAEB33FBC3EC33FCED33FD7E0A91C0
:100CF000F68B618A6022C3EC9EFCED9400FDC3EC90
:100D00009AFCED9BFDC3EC9423ED940050047C23EE
:100D10007D00C3EC94FFED940140047CFF7D017BDA
:100D2000FF0B7A000AEA7009C3EC33FCED33FDA136
:100D300021EC8AF0A4AEF0ED8AF0A42E947C40E47D
:100D4000EAF460DD22D23691901205A31205A37A4F
:100D5000007B007C1012059BE5542AFA74003BFBD3
:100D6000DCF37C04C3EB13FBEA13FADCF7FFEB6064
:100D7000027FFFC23691902278A5E6F954037000F5
:100D8000E9540C7000E954307000E954C07000223E
:100D90007567007568007597DE7597AD7581C043FE
:100DA000FF8075EF0675A90071807580FF75F1F001
:100DB00075A4007580FF75D4FF75902A75F23F7594
:100DC000A53F75902A75D53F75A60175E34075E27C
:100DD000027180E4F8F6D8FD7190121413789886A9
:100DE00064753001C2AF1205AB711D1205A37123EA
:100DF0001205A371291205A3B178C2AF75670075FA
:100E0000680078FA79FA308507D9FBD8F7021C0018
:100E10009122919078988664718075A91375A710B6
:100E200075C10075A70075660075E40575881175B4
:100E30008E0475890975C80475910475D84075D9F3
:100E40000875F782759E0375960075DA4275DB4268
:100E500075A82375E69075B801759B80759D007522
:100E6000D10C75BCB975BB1075E88075B20112055F
:100E700097D2AF753C00C2301205ABC231C232C24C
:100E800033C2347552007553007522001205A7C392
:100E9000E522940A5002E160D2317522001205A7C2
:100EA000C3E522940A5002E160C231D232752200B9
:100EB0001205A7C3E522940A5002E16075E4D575D6
:100EC0008851758E017589AA758C00758D00C2A92F
:100ED000D2ABD2AA756B80756A14756E50C232D2CD
:100EE0003475220A1205A7756A10C3E522940A75A3
:100EF00052007553004069758E0C756B00756A2839
:100F0000756E2875220A1205A7756A20C3E522941A
:100F10000A7552007553004047758E0C756B8075CD
:100F20006A14756E1475220A1205A7756A10C3E556
:100F300022940A755200755300402575E4057588A2
:100F400011758E04758909D2A9C2ABC2AAC234D266
:100F5000337522001205A7C3E522940A4002A1FAC4
:100F600012059B203003020DFAC2AF711D711D7175
:100F70001DD2AF1205AB203403303A0302101F120A
:100F8000059B788CE6C39401500302101FE530C323
:100F90009401500302101F7567A57568F17F02D296
:100FA0003691901205A7C2AFC2369190C3E5549412
:100FB0007FD2AF406A120597C2AF712FD2AFDFDF89
:100FC000B145C3EF7897F61205AB1215007F0AD230
:100FD0003691901205A7C2AFC2369190C3E55494E2
:100FE0007FD2AF50E8120597C2AF711D12059F71F5
:100FF0001DD2AFDFDAB145EF24037896F6F8799782
:10100000E7C394234003985006E824237897F61208
:1010100005AB915AB12F1205A7120C90020DFA756B
:1010200067007568001205A7C3E5549401400302E8
:101030000F76C2AF120B2F120B2F120B2FD2AF1243
:1010400005AB753000E4F537F5380537E537F47052
:101050003F0538789AE67819146012783214600DDA
:10106000787D14600878FA146003753800C3E53899
:1010700098401D120B801205971538753700789926
:101080008664C2AF120B2FD2AF789886641205A780
:1010900012059FE5237003020DFAC3E55494015035
:1010A0000AC3E5529401501602104A1205A7E5231F
:1010B0007003020DFA755200755300021260C3E509
:1010C0005294017017C2AF120B8078998664120B8C
:1010D0001D78988664D2AF1205A74152C3E5529499
:1010E000027017C2AF120B8078998664120B2378B6
:1010F000988664D2AF1205A74152C3E5529403709B
:1011000017C2AF120B8078998664120B29789886E3
:1011100064D2AF1205A74152C3E55294047017C2BE
:10112000AF120B8078998664120B2F78988664D260
:10113000AF1205A74152C3E55294057017C2AF1212
:101140000B8078998664120B2F78988664D2AF1240
:1011500005A74152C3E55294077019C3E55394069D
:101160005002019A7401303A0274037888F6C2384A
:10117000C2394152C3E55294087019C3E55394062D
:101180005002019A7402303A0274047888F6D23818
:10119000D2394152C3E55294097017C3E5539406FE
:1011A0005002019A303A0BC37888E69402F6C23AAC
:1011B0004152C3E552940A7016C3E5539406500297
:1011C000019A203A0A7888E62402F6D23A4152C3BC
:1011D000E55294147025C3E55394065002019AC257
:1011E000AF901A0B740093D2AF7888F613C238C24E
:1011F000394002D2384002D2398057C3E5529415A3
:101200007038C3E5539406404FC2AF901A0B740078
:1012100093D2AFF8B801027402B802027401B803A5
:10122000027404B8040274037888F613C238C23911
:101230004002D2384002D2398018C3E552940C7073
:10124000117567A57568F1C3E5539406400A915A74
:10125000D2AF755200755300756700756800019A2A
:10126000C2AF120B80E4D2AFE4F55EF524F525F5AC
:101270003D755E0812059712060030EDFDA8BDA968
:10128000BEE97001F8885F120604755E08C2AF12ED
:10129000066B855D5B855D5CD2AF75A71075C1304F
:1012A00075A70075A903756601303A07C238303555
:1012B00002D238D228753900120AD8120AFB120657
:1012C0007A12068112067A12068112067A1209062D
:1012D000120A04120A4C1206811208F6202C03127C
:1012E00005BA302C031205EA120A04120A6F12061C
:1012F00081120906120A04120A921206811208F6D5
:10130000120A04120AB5120681120906120A041200
:101310000AD81206811206001208F6120A04120AEE
:10132000FB120604120681302827855D5B79187A46
:101330000CC3E53999400EC228D2298A3B855D5BF2
:10134000855D5C800CC3E554940140030212CD61BD
:10135000D730291F202B1CE53B147006C229D22A46
:1013600041CDF53B203A07C3E554940140030212F6
:10137000CD8064753C00203A0F78FA79A4E76002CA
:101380007803C3E55598504FE523604B303A17205A
:101390003805203507800F303502800A202B07D210
:1013A0002B855D5B41FD78F0302B05855D5B7820FA
:1013B000C3E5489850030212CD302B1BC22BC23814
:1013C000303502D238D229753B12855D5B41CD059F
:1013D0003CE554600261DA753C00C2AF120B8075C7
:1013E000240075250075A91375A71075C10075A790
:1013F00000756600D2AF1205A7120B8078A4E660D4
:1014000006C291C293C295C3E53C94044003020D09
:10141000FA0145901A0D78209193E520B4550AA35E
:101420009193E520B4AA0280137567A57568F1123F
:101430000B90915A756700756800801D901A0378AB
:10144000807B0A9193A308DBFA901A0F788C7B1AA1
:101450009193A308DBFA901A2922C2AF91D691B3D7
:10146000901A0074109198A374079198A374219115
:1014700098901A0378807B0A9197A308DBFA901A58
:101480000F788C7B1A9197A308DBFA91E991C790AA
:101490001A2922E493F622E6438F01538FFDFFC3FE
:1014A000E583941C400122EF8567B78568B7F05348
:1014B0008FFE22438F02438F018567B78568B790FF
:1014C0001A0DF0538FFC22901A0D74559198901AB2
:1014D0000E74AA9198227A3079D07820901A40918F
:1014E00093E520F709A3DAF7227A3079D0901A40F1
:1014F000E7919809A3DAF9227C051205ABDCFB22FF
:10150000C2AF120B1D120B23120B29120B2F120547
:101510009F120B1D120B23120B29120B2F12059F6A
:10152000120B1D120B23120B29120B2FD2AF22C24A
:10153000AF120B2F120B29120B23120B1D12059F3A
:10154000120B2F120B29120B23120B1D12059F12C7
:0E1550000B2F120B29120B23120B1DD2AF22F0
:1019FD00020D90100721FFFFFFFFFFFF09FF01FF01
:101A0D0055AA01FFFFFFFFFF03FFFFFF25D0285061
:0D1A1D0004FF02FF7AFF0701FFFF0000FF3A
:101A4000234F5F485F373023202020202020202094
:101A500023424C48454C492445464D3842323123B7
:101A60002020202020202020202020202020202076
:101C0000C2AFC2D37597DE7597AD7581C075A90057
:101C100043FF80752438752503B1DB7529A5752A26
:101C2000F143F12053A4DFD28575D4FF75E3407DE5
:101C3000FA780379E67C10752200752300901DE880
:101C40007B0675249875250130850281482085081A
:101C5000D8FBD9F9DCF781BA308508D8FBD9F9DC93
:101C6000F781BAB19BE493A3C39A6004DDC381BA40
:101C7000DBDBB18D600281317B08E493FAA3B16EA6
:101C8000DBF87A30B16E752200752300B18DEAFC65
:101C9000EBFDC3ED94FE400EB18D8A278B28ED300D
:101CA000E0048A828B83B18D7AC270D8C3ED94FE32
:101CB000601950CEBD0029EC600F7520007521FF22
:101CC000752900752A000200008100A827A92808AC
:101CD00009D804D90281DDB191EAF281D10D81A642
:101CE000C3ED94035051EDA2E092007AC5C3E582A2
:101CF0009400E583941C508C200010438F02438F86
:101D0000018529B7852AB7F0300027A827A9280818
:101D100009438F01538FFDD804D902A132C3E58353
:101D2000941C4003A3A117E28529B7852AB7F0A325
:101D3000A117538FFC81827AC1BD030CE493A3FAEF
:101D4000B152DCF8B14A81828184AA22AB23B16E00
:101D5000EBFAEA6222752608C3E52313F523E52290
:101D600013F52250066323A0632201D526EAB1DBD6
:101D7000B1DB75260AEAF4200102D285300102C2E5
:101D800085B1DBC3134002C201D526EB22B191EA33
:101D9000FB208502A191308502A196752608AE240C
:101DA000AF25C3EF13FFEE13FEB1DFB1DBC3EA13C0
:101DB0003085024480FA30E703632201C3E5231330
:101DC000F523E52213F52250066323A0632201D5F3
:101DD00026D9E52265236523F52222AE24AF250E00
:101DE0000FDEFEDFFCD20122424C48656C693437BD
:061DF0003164E8B20601B7
:00000001FF
